:100000000C9437000C945E070C945E070C945E070A
:100010000C945E070C945E070C945E070C94DA0651
:100020000C945E070C945E070C940D040C949604DB
:100030000C945E070C945E070C943D050C945E07CF
:100040000C94F8050C945E070C945E070C945E0704
:100050000C945E070C945E070C945E070C945E078C
:100060000C945E070C945E0701000130800011249F
:100070001FBECFEFD8E0DEBFCDBFE8E6F0E040E046
:1000800017C0B591A59135912591059107FD0CC03B
:1000900095918591EF01F92FE82F05900D92A21708
:1000A000B307D9F7FE0104C01D92A217B307E1F709
:1000B000ED36F40731F70E9461000C945F00F8946C
:0200C000FFCF70
:1000C2000E947E028091010190910201892B71F0C0
:1000D2008BB18F7B8BB90E945407EEE6F0E08081F2
:1000E2008D7F808380818E7F80837DC1809100019E
:1000F200882309F478C1109200018091090190913E
:100102000A01A0910B01B0910C0180930D01909313
:100112000E01A0930F01B093100180910D019091F7
:100122000E01A0910F01B0911001880F991FAA1F13
:10013200BB1F880F991FAA1FBB1F880F991FAA1FD9
:10014200BB1F880F991FAA1FBB1F880F991FAA1FC9
:10015200BB1F880F991FAA1FBB1F80930D0190938D
:100162000E01A0930F01B093100180912501882305
:1001720031F080911301909114010E94BF0580918A
:100182002A0190912B0180349105E9F0811521E03B
:10019200920721F0089709F047C02EC080910D0107
:1001A20090910E01A0910F01B0911001892F9A2F09
:1001B200AB2FBB2780930D0190930E01A0930F01EB
:1001C200B093100131C080910D0190910E01A09168
:1001D2000F01B0911001689415F8B695A7959795FF
:1001E20087951694D1F780930D0190930E01A093F9
:1001F2000F01B093100118C080910D0190910E0172
:10020200A0910F01B0911001689412F8B695A795CC
:10021200979587951694D1F780930D0190930E01CF
:10022200A0930F01B09310012091050130910601B6
:10023200409107015091080160910D0170910E01EA
:1002420080910F01909110010E941F0760930D0190
:1002520070930E0180930F019093100180910D0114
:1002620090910E01A0910F01B09110019F5FAF4FCD
:10027200BF4F80930D0190930E01A0930F01B09395
:10028200100180910D0190910E01A0910F01B0918A
:100292001001072E79E0B695A795979587957A95DF
:1002A200D1F7702D80930D0190930E01A0930F0151
:1002B200B093100180910D0190910E01A0910F0158
:1002C200B0911001805C9F4FAF4FBF4F80930D01E3
:1002D20090930E01A0930F01B093100180910D0134
:1002E20090910E01A0910F01B0911001689416F83F
:1002F200B695A795979587951694D1F780930D019A
:1003020090930E01A0930F01B093100180910D0103
:1003120090910E01A0910F01B091100180930D01F7
:1003220090930E01A0930F01B093100180910D01E3
:1003320090910E01A0910F01B0911001892F9A2F77
:10034200AB2FBB2790931E0180931D018091250145
:100352008823E1F085B1806285B985B18F7D85B949
:100362001092250180911D0190911E01909304012C
:100372008093030180911301909114010E94BF05A3
:10038200EEE6F0E080818160808316BC80910D01F1
:1003920090910E01A0910F01B091100199279093B5
:1003A2001201809311018091130190911401019720
:1003B200D1F48091110190911201C29738F482E335
:1003C20090E090931201809311010DC08091110170
:1003D20090911201893C910530F088EC90E0909365
:1003E20012018093110130996DCE8BB18F7B8BB945
:1003F20080912A0190912B0190931801809317010B
:10040200E1EBF0E08081877F8083A0EBB0E08C910C
:1004120082608C938C918E7F8C938CE98093B30055
:10042200A0E7B0E08C9182608C93808184608083AD
:1004320080818260808380818160808388EE93E006
:100442009093200180931F018091210190912201BC
:10045200A0912301B091240190931A018093190174
:10046200109216011092150136C0809119019091D7
:100472001A0160911F01709120010E940B07CB01AC
:100482000E943E078091190190911A0160911F010B
:10049200709120010E940B0790931A018093190119
:1004A20020911F0130912001ADECBCEC0E942F077E
:1004B2009695879596958795969587959093200121
:1004C20080931F01809115019091160101969093DE
:1004D20016018093150180911501909116010497E0
:1004E20020F280911701909118010E94BF05E0E768
:0A04F200F0E080818D7F8083E5CD6E
:1004FC0084B1806284B985B18F7D85B98FB78068EE
:10050C008FBF81E090E090930201809301013099BC
:10051C00A9C0E1EBF0E08081877F8083A0EBB0E0A5
:10052C008C9182608C938C918E7F8C938CE98093D0
:10053C00B300A0E7B0E08C9182608C9380818460E2
:10054C00808380818260808380818160808310922F
:10055C00B20010922F0110922E0180912E019091D9
:10056C002F01883C9105C8F310922D0110922C019B
:10057C0088EE93E09093200180931F011092160156
:10058C001092150136C00E94F30640911F01509144
:10059C00200180911B0190911C01489F9001499F63
:1005AC00300D589F300D112480912C0190912D010C
:1005BC00820F931F90932D0180932C0120911F018A
:1005CC0030912001ADECBCEC0E942F0796958795DD
:1005DC0096958795969587959093200180931F010A
:1005EC0080911501909116010196909316018093BC
:1005FC0015018091150190911601049720F28091BC
:10060C002C0190912D019093260180912C019091B9
:10061C002D018093290185B18F7D85B9F894F999C5
:10062C00FECF12BC11BC8091260180BD8FB38F7D93
:10063C008FBB8FB38F7E8FBBFA9AF99A7894F8940C
:10064C00F999FECF12BC81E081BD8091290180BD5A
:10065C008FB38F7D8FBB8FB38F7E8FBBFA9AF99A36
:10066C007894FFCFE0E8F0E080818F778083808101
:10067C008F7B808380818F7D808380818F7E808340
:10068C00A1E8B0E08C918F7E8C938C91877F8C93BA
:10069C0080818D7F808380818E7F80838C91806828
:1006AC008C938C9180648C9380E09DE7909389006F
:1006BC0080938800EFE6F0E0808180628083808107
:1006CC008260808380E091E00E94F80481E090E0F9
:1006DC009093280180932701EEE6F0E080818D7FD6
:1006EC00808380818E7F80838AB180648AB98BB14C
:1006FC008F7B8BB9F894F999FECF12BC11BC8FB3D8
:10070C0081608FBB80B5809326017894F894F99919
:10071C00FECF12BC81E081BD8FB381608FBB80B5F1
:10072C008093290178948091260190E0A0E0B0E0BC
:10073C008093210190932201A0932301B093240173
:10074C008091210190912201A0912301B09124016B
:10075C00BA2FA92F982F88278093210190932201DB
:10076C00A0932301B09324012091290180912101B0
:10077C0090912201A0912301B0912401820F911D2F
:10078C00A11DB11D8093210190932201A0932301FF
:10079C00B09324018091210190912201A091230119
:1007AC00B0912401843F9140A105B10568F080917E
:1007BC00210190912201A0912301B0912401813D4E
:1007CC009740A105B10560F088EE93E0A0E0B0E0A1
:1007DC008093210190932201A0932301B0932401D3
:1007EC00209121013091220140912301509124014B
:1007FC0060E070ED87E090E00E94B8062093050160
:0E080C003093060140930701509308010895B0
:10081A001F920F920FB60F9211242F933F934F936B
:10082A005F936F937F938F939F93AF93BF93EF934E
:10083A00FF93109285001092840080912701909175
:10084A002801892B29F0109228011092270158C0FB
:10085A0080918600909187008C369740F0F48091C1
:10086A001301909114018034910569F0811521E0FA
:10087A00920721F0089709F043C00AC080E490E08B
:10088A000E94F8043DC088E090E00E94F80438C055
:10089A0081E090E00E94F80433C080918600909134
:1008AA008700A0E0B0E08093090190930A01A09329
:1008BA000B01B0930C01A0911301B0911401209186
:1008CA00090130910A0140910B0150910C010E94DB
:1008DA0049076093090170930A0180930B01909371
:1008EA000C018091010190910201892B49F010922B
:1008FA0002011092010181E0809300018093250199
:10090A00FF91EF91BF91AF919F918F917F916F91DD
:10091A005F914F913F912F910F900FBE0F901F90B3
:02092A0018951E
:10092C001F920F920FB60F9211242F933F934F9358
:10093C005F936F937F938F939F93AF93BF93EF933B
:10094C00FF93109285001092840081E090E09093C8
:10095C0028018093270190930201809301018091DB
:10096C001301909114018115914051F48BB18F7B3F
:10097C008BB981E090E0909302018093010121C03A
:10098C0080911301909114018034910529F480E039
:10099C0091E00E94F80415C080911301909114010C
:1009AC00089729F480E490E00E94F8040AC0809132
:1009BC00130190911401019721F488E090E00E94BA
:1009CC00F804FF91EF91BF91AF919F918F917F911F
:1009DC006F915F914F913F912F910F900FBE0F90A0
:0409EC001F901895AB
:1009F000109285001092840090931401809313014B
:100A00008830910511F118F4019759F10895803457
:100A1000910579F08115914079F5E1E8F0E0808168
:100A20008460808380818D7F808380818E7F8083BE
:100A30000895E1E8F0E080818B7F8083808182608F
:100A400080838081816080830895E1E8F0E0808187
:100A50008B7F808380818260808380818E7F808392
:100A60000895E1E8F0E080818B7F808380818D7F35
:0A0A700080838081816080830895F7
:100A7A001F920F920FB60F9211242F933F934F9309
:100A8A005F936F937F938F939F93AF93BF93EF93EC
:100A9A00FF93EEE6F0E080818D7F808316BC808133
:100AAA00816080835E990DC08BB180648BB981E0CF
:100ABA008093000180911301909114010E94BF0557
:100ACA0003C08BB18F7B8BB980911D0190911E0160
:100ADA009093040180930301FF91EF91BF91AF912D
:100AEA009F918F917F916F915F914F913F912F913C
:0A0AFA000F900FBE0F901F9018958B
:100B040020E030E041E050E034C085B1806285B936
:100B14001092B20010922F0110922E0104C030994D
:100B240002C021E030E080912E0190912F018436A3
:100B34009105A8F385B18F7D85B91092B20010920A
:100B44002F0110922E0104C0309902C021E030E040
:100B540080912E0190912F0184369105A8F32115DF
:100B6400310529F050931C0140931B0108954F5FF8
:0A0B74005F4F4A30510548F2089522
:100B7E0090932B0180932A0188309105F1F018F49F
:100B8E00019729F108958034910569F081159140FE
:100B9E0039F585B5846085BD85B58D7F85BD85B5F7
:100BAE008E7F85BD089585B58B7F85BD85B58260A9
:100BBE0085BD85B5816085BD089585B58B7F85BD65
:100BCE0085B5826085BD85B58E7F85BD089585B559
:100BDE008B7F85BD85B58D7F85BD85B5816085BDD6
:020BEE00089568
:100BF0001F920F920FB60F9211248F939F93EF9332
:100C0000FF9385B1806285B985B18F7D85B980916B
:100C100003019091040101979093040180930301D3
:100C20008091030190910401892B81F485B3826046
:100C300085BBEEE6F0E080818E7F8083809111019C
:100C40009091120187BD808182608083FF91EF9136
:0E0C50009F918F910F900FBE0F901F901895DF
:100C5E0085B1806285B91092B20010922F01109268
:100C6E002E0120E030E004C0309902C021E030E0D7
:100C7E0080912E0190912F010A97B0F385B18F7D4F
:100C8E0085B91092B20010922F0110922E0104C05D
:100C9E00309902C021E030E080912E0190912F0119
:100CAE0084369105A8F3232B21F010921C0110928B
:040CBE001B01089579
:100CC2001092B20085B18F7D85B910922F011092DA
:100CD2002E0180912E0190912F0184369105C8F347
:100CE2001092B20085B1806285B910922F011092E4
:100CF2002E0180912E0190912F010A97D0F310922C
:100D0200B20085B18F7D85B910922F0110922E010C
:0E0D120080912E0190912F01C297D0F3089589
:100D2000AC0122C01092B20095B1906295B91092B8
:100D30002F0110922E0120912E0130912F0122338C
:100D40003105C8F31092B20095B19F7D95B910920C
:100D50002F0110922E0120912E0130912F0122336C
:100D60003105C8F34150510941155105D9F608958F
:100D7000A1E21A2EAA1BBB1BFD010DC0AA1FBB1F9F
:100D8000EE1FFF1FA217B307E407F50720F0A21B11
:100D9000B30BE40BF50B661F771F881F991F1A947E
:100DA00069F760957095809590959B01AC01BD01A8
:040DB000CF010895D2
:100DB4001F920F920FB60F9211248F939F9310924C
:100DC400B20080912E0190912F01019690932F01F2
:100DD40080932E019F918F910F900FBE0F901F90C3
:020DE400189560
:100DE60084E690E090931C0180931B010E942F06DD
:100DF60080911B0190911C01892B11F00E948205A4
:100E060080911B0190911C010A9708F0FFCF08956D
:100E1600AA1BBB1B51E107C0AA1FBB1FA617B7071A
:100E260010F0A61BB70B881F991F5A95A9F7809536
:080E36009095BC01CD01089567
:100E3E00DB018F939F930E944907BF91AF91A29FB1
:100E4E00800D911DA39F900DB29F900D11240895BA
:100E5E00A29FB001B39FC001A39F700D811D1124ED
:0E0E6E00911DB29F700D811D1124911D0895DC
:100E7C00CF93DF93EC010E946106CE010E94900695
:060E8C00DF91CF910895F3
:100E92000E942F07A59F900DB49F900DA49F800DD7
:060EA200911D11240895CA
:100EA80085B58B7F85BD85B58D7F85BD85B58E7FE5
:040EB80085BD089557
:040EBC000C94000092
:00000001FF
